:101107002025322E582000257300205379737465EB
:101117006D2048414C54454400204C6F632E2053AA
:10112700746570706572206572726F7200205379F2
:101137007374656D20524553455400202E2E2E2082
:101147005361766500202E2E2E2045646974004376
:101157006C6173736963616C20536875747465722D
:10116700202E2E2E00202020202E2E2E20506C6583
:10117700617365207761697400456E68616E6365A8
:10118700642053687574746572202E2E2E002042D9
:10119700617365202025332E64202D203078255853
:1011A7002020002052616E6765202573205B565D05
:1011B70000202563202D20257300204E6F742041C9
:1011C7007661696C61626C65202E2E2E0020466167
:1011D70064696E67202025332E64205B735D2020B1
:1011E7000020456E61626C6564200020446973616C
:1011F700626C65640020436F6E6669726D205245AC
:101207004C4F4144202E2E2E00202E2E2E204C6F88
:101217006164656400204C4F47202D2025322E64E1
:101227000020536F6674205265736574202E2E2E2E
:1012370000202D2D3E2020506C656173652057617D
:10124700697400202E2E2E2053656C656374002070
:101257002E2E2E2045646974202000202E2E2E204D
:1012670043616E63656C20496E70757400202E2E85
:101277002E20466C6173682050726F63657373002C
:1012870047524159205343414C45205348555454E4
:1012970045520056657273696F6E20312E383000E3
:1012A700504547415355532039392E2E30310020B0
:1012B7005344785020434F4D4D206572726F720032
:1012C700494E4954206279706173736564002573D0
:1012D7002025342E3166202D20256420256320000B
:1012E70020446D782025332E64202D2025322E644E
:1012F7002025322E6420200020416E616C6F67200C
:1013070025322E6420252520002046616465202D86
:101317002025322E64205B735D2000204D616E75A1
:10132700616C20636F6E74726F6C20000000002088
:1013370052656D6F746520636F6E74726F6C2000F9
:1013470000000020362E32350020372E35300020A1
:10135700382E37350031302E30300031312E3235CE
:10136700002047343035202F5043532020200000E1
:1013770000000000002047343035202F5043532D04
:101387004949000000000000004C6F6E672066614D
:101397006465200000004469726563742020202082
:1013A7000000002043757276652041202020202010
:1013B70020202020002043757276652042202020BF
:1013C70020202020202000205043532D4920636FE8
:1013D7006D70617469626C6500204C696E6561723D
:1013E7002074726176656C202020000304050607CF
:1013F70008090A0F14191E2328323C4F70657261C1
:1014070074696F6E206D6F646520000000000044F2
:101417004D5820616464726573732020202000009A
:10142700000000414443207363616C696E672020AC
:101437002020000000000053687574746572205402
:1014470079706520202000000000005368757474CF
:1014570065722044796E616D696300000000004485
:10146700696D6D657220436F6E74726F6C2000003A
:10147700000000436861726163746572697374691F
:10148700632000000000004D616E75616C204661AD
:1014970064696E672020000000000041636F757368
:1014A70074696320626565702020000000000052A7
:1014B700656C6F61642064656661756C74730000A8
:1014C7000000004572726F7220436F6465732020BD
:1014D70020200000000000446961676E6F73746923
:1014E70063732020202000000000004D616E7561AD
:1014F7006C0052656D6F74650020204E6F20726519
:1015070063657074696F6E004E6F2044494D4D4599
:1015170052206461746100202020446D782064614A
:061527007461204F4B002F
:062F2700C10EC110C10F34
:101E1800FF7B007A00798A2208F6FF798AE718267C
:101E28002F788DF622AF68EF3395E0FE74F22FF528
:101E38008274133EF583E49322AF32EF3395E0FECC
:101E48007C007D14020664AF03AE020206647B4484
:101E58007A07E4FD7FC022E4FBFAFD7FC022D2F8B6
:101E6800D2F9A2F8B322E5332BFFE5323A2292F8F1
:101E7800D2F9C2F922C3E56A9401E569940022C245
:101E8800F87F017E0022E56475F00AA4FBAAF0221F
:071E9800753707753844227D
:052F2E00D2F8D2F922E7
:082027008F448B458A4689476E
:10202F00C2F8120049C2F9E54425E054FEF544E434
:10203F00FFE54425E0F544121E760FBF08F3121E8C
:10204F00669207C2F9200602D20730073AE54860C8
:10205F0036AB45AA46A94712060CFEE4FFEE25E073
:10206F00FE121E760FBF08F5121E669207C2F97494
:10207F00012547F547E43546F5461548200602D2B7
:10208F0007D2AED2BE80C3C2F8D2F9120049D2F83D
:02209F00A20796
:0120A100221C
:081C6B008F438B448A45894632
:101C7300E4F549754A80C2F8120049C2F9E54325E3
:101C8300E04401F543E4F548E54325E0F543121E3E
:101C9300760548E548B408F0121E669205C2F9308D
:101CA3000550E547604CE4FFF548D2F930F804E508
:101CB3004A4207C2F9E54AC313F54A0548E548B461
:101CC30008E8AB44AA45A946EF1206521547E54773
:101CD3006004C2F88002D2F8D2F9120049C2F97442
:101CE300012546F546E43545F5450549D2AED2BE54
:0D1CF30080ADC2F8D2F9120049D2F8AF4915
:011D000022C0
:102C1D00C20575430A788AA60708A60520051CE596
:102C2D004360187F017E00120003121E19754802C1
:0D2C3D00D2067F50122027920580E1A205EB
:012C4A002267
:102B8600C20475340A788AA607ECFF3395E0EF088D
:102B9600F6ED08F620041CE53460187F017E00126D
:102BA6000003121E19754803D2067F501220279281
:052BB6000480E1A2040F
:012BBB0022F7
:102E0700788AA607121E19754801D2067F5012202C
:102E170027121E197547017F50121C6B788AE6FF2F
:012E27002288
:022988008F14AA
:10298A00788AA614121E191229C8121E197547012F
:10299A007F50121C6B788AE6F515E51404F6121EB0
:1029AA00191229C8121E197547017F50121C6BE5AE
:0D29BA0015FE788AE67C002400FFEC3EFE4E
:0B29C70022754801D2067F5002202735
:052F3300D2FBD2FC22DC
:0429D2008F348D357C
:1029D600E5356030A834E6F537753608E536601714
:1029E600E53725E0F537153692FBC2FCD2FC7F644D
:1029F6007E00122CA380E5053415357F647E001217
:102A06002CA380CCD2FBD2FC7FF47E01122CA33007
:052A1600FB02C322D306
:012A1B002298
:1028F20075357820940BA20492057F0A7E00122B74
:102902004E43E80FD2EED2ECE5E8540FF534300333
:102912001D20941AE535600B7F0A7E001200031514
:102922003580EED2057F0A7E00122B4E80E3C2EE86
:0A293200C2ECC2C1C20ED2B9AF342C
:01293C002278
:102D710075337820941AE533600B7F0A7E001200C8
:102D810003153380EED2057F0A7E00122B4E80E3BD
:062D9100C2C1C20ED2B95E
:012D97002219
:0D2F02003094097F017E0012000380F4224C
:022A1C008F40E9
:102A1E007F30122E078F41E5412431FFAD40122C3D
:102A2E001D0541E541C3940550028001C34003E4F6
:102A3E00F541AD417F30122C1DE4F542D2057F1ECB
:102A4E007E00122B4E7FC87E001200030542E54227
:052A5E00C3940640E7EF
:012A63002250
:1027F3007F30122E078F341534E4F535E534C39456
:102803000550028001C34003753404E5342431FFCD
:10281300122E0774362535F8A60715340535E53528
:10282300C3940540D7E4F5357BFF7A1179077436F5
:102833002535F8E6754300F544120CFA0535E53500
:05284300C3940540E311
:01284800226D
:102E2800E4FD7F30122C1DE4F533E5332431FF7DBA
:0D2E3800FF122C1D0533E533C3940540ED5A
:012E4500226A
:102B15008B328A338934122E947F40122EBF853230
:102B2500438533448534457BFF7A11790E120CFABF
:102B35007F14122EBF7BFF7A117911120CFA7FF2E6
:092B4500122A1CD2AED2BE80FAA5
:102BEE00122E947F40122EBF7BFF7A117920120C89
:102BFE00FA7F14122EBF7BFF7A117934120CFA7FF2
:0F2C0E00F1122A1CD2057FD07E07122B4E80FEBA
:041F23008F328D3339
:101F2700753405753505C202788A7680087681088A
:101F37007682798AE718262482788DF6200241E591
:101F470035603DE532C3134533121E18754804D278
:101F5700061220274011E534600DD2057F0A7E0066
:101F6700122B4E153480DC7F907E01122CA320F9B2
:101F770004D20280077F327E00120003153580BC31
:101F87007FC87E00120003E5346006E5356002D3A2
:0E1F970022D2057FD07E07122B4E122BEEC3F6
:011FA5002219
:081E9F008F368D378A388B392C
:101EA700753A05753B05C202788A7690E538FF33A7
:101EB70095E0EF08F6AF39E539121E20200241E51B
:101EC7003B603DE536C3134537121E18754804D2EB
:101ED700061220274011E53A600DD2057F0A7E00E1
:101EE700122B4E153A80DC7F907E01122CA320F92D
:101EF70004D20280077F327E00120003153B80BCAC
:101F07007FC87E00120003E53A6009E53B6005AE35
:0B1F170038AF3922122BEE7EFF7FFF57
:011F2200229C
:042198008F368D37BA
:10219C00753A05753B05C202788A76A008A6030835
:1021AC00A639798AE718262539788DF6200241E57B
:1021BC003B603DE536C3134537121E18754804D2F3
:1021CC00061220274011E53A600DD2057F0A7E00E9
:1021DC00122B4E153A80DC7F907E01122CA320F935
:1021EC0004D20280077F327E00120003153B80BCB4
:1021FC007F647E00120003E53A6006E53B6002D383
:05220C0022122BEEC3BD
:0122110022AA
:041D8D008F368D37C9
:101D9100753C05753D05C202788A76C0AE02AF0377
:101DA1007C007D641206CB788BA607AE3AAF3B7CF4
:101DB100007D641206CB788CEFF6121E23200241BF
:101DC100E53D603DE536C3134537121E18754804DD
:101DD100D2061220274011E53C600DD2057F0A7E14
:101DE10000122B4E153C80DC7F907E01122CA3202B
:101DF100F904D20280077F327E00120003153D8074
:101E0100BC7F647E00120003E53C6006E53D600294
:061E1100D322122BEEC3E8
:011E170022A8
:042212008F368D373F
:10221600753B05753C05C202788A76B008A603E5CB
:1022260039C313E53A13FF08F6121E23200241E5CF
:102236003C603DE536C3134537121E18754804D277
:10224600061220274011E53B600DD2057F0A7E006D
:10225600122B4E153B80DC7F907E01122CA320F9B9
:1022660004D20280077F327E00120003153C80BC38
:102276007F647E00120003E53B6006E53C6002D306
:0522860022122BEEC343
:01228B002230
:04228C008F368D37C5
:10229000753A05753B05C202788A76D008A6030810
:1022A000A639798AE718262539788DF6200241E586
:1022B0003B603DE536C3134537121E18754804D2FE
:1022C000061220274011E53A600DD2057F0A7E00F4
:1022D000122B4E153A80DC7F907E01122CA320F940
:1022E00004D20280077F327E00120003153B80BCBF
:1022F0007F647E00120003E53A6006E53B6002D38E
:0523000022122BEEC3C8
:0123050022B5
:042306008F368D374A
:10230A00753805753905C202788A76E0EA08F6AFAB
:10231A0003EB08F6121E23200241E539603DE5363B
:10232A00C3134537121E18754804D20612202740D7
:10233A0011E538600DD2057F0A7E00122B4E153842
:10234A0080DC7F907E01122CA320F904D202800740
:10235A007F327E00120003153980BC7F647E001232
:10236A000003E5386006E5396002D322122BEEC37A
:01237A002240
:0420A2008F368D37B1
:1020A600753805753905C203788A7620300204E64C
:1020B6004401F6788B76AA0876BB798AE718262437
:1020C600BB788DF6200341E539603DE536C31345FF
:1020D60037121E18754804D2061220274011E5381B
:1020E600600DD2057F0A7E00122B4E153880DC7FEC
:1020F600907E01122CA320F904D20380077F327E42
:1021060000120003153980BCE5386006E539600227
:06211600D322122BEEC3E0
:01211C0022A0
:081FA6008F338D348A358B3630
:101FAE00753905753A05C203D3E5369538E535958D
:101FBE00374006853735853836788A7638E53508E0
:101FCE00F6AF36E536121E20200341E53A603DE5B8
:101FDE0033C3134534121E18754804D20612202737
:101FEE004011E539600DD2057F0A7E00122B4E1589
:101FFE003980DC7F907E01122CA320F904D203805D
:10200E00077F327E00120003153A80BCE53A600568
:08201E00AE35AF3622122BEEA5
:012026002297
:041A13008F368D3746
:101A1700753E05753F05C204E53B2BE53A3AC3948D
:101A2700005009C3E49BF53BE49AF53AE53B2BFFED
:101A3700E53A3AFED3EF953DEE953C400AE53D9BEE
:101A4700F53BE53C9AF53AD3E53B9400E53A6480EB
:101A570094804008788A7611D2038006788A7610B7
:101A6700C203300206788AE64404F6AF3BAE3A1268
:101A77002ED28E3A8F3BE53B453A6075E53AFF3308
:101A870095E0EF788BF6AF3BE53B121E2020044133
:101A9700E53F603DE536C3134537121E1875480408
:101AA700D2061220274011E53E600DD2057F0A7E3F
:101AB70000122B4E153E80DC7F907E01122CA32056
:101AC700F904D20480077F327E00120003153F809D
:101AD700BCE53F60197F037E00120003300305AEAB
:101AE7003AAF3B22C3E4953BFFE4953AFE22022B33
:051AF700EE7E007F00FF
:011AFC0022C7
:10169300300341AD6AAC697F10122B86AD667F23A0
:1016A300122C1DAD607F20122C1DAD617F24122CE6
:1016B3001DAD627F22122C1DAD677F26122C1DAD3E
:1016C300687F28122C1DAD657F29122C1DAD637F09
:1016D30021022C1D7F10122E07EF7F00FEC006C0D3
:1016E300077F11122E07EFFDD0E02DF56AD0E0340D
:1016F30000F569121E7D400BD3E56A94F9E5699400
:10170300014006756900756A017F23122E078F66F3
:10171300D3E566648094815009C3E5666480948050
:101723005003E4F5667F20122E078F60E560D394A3
:10173300055007E560C3940150037560057F2412CB
:101743002E078F61E561D394025007E561C39401CD
:1017530050037561027F26122E078F67D3E56764F6
:101763008094845009C3E56764809481500375674E
:10177300017F27122E078F64E564D394BA5007E5DF
:1017830064C39400500375640A7F28122E078F6880
:10179300D3E5686480948F5009C3E56864809480BE
:1017A30050037568037F291217C1F5657F2112174E
:1017B300C1F5637F22122E07EF5401F56222122E28
:0517C30007EF540122B4
:10002600300207AD647F27022C1D7F27122E078F13
:1000360064E564D394BA5007E564C394005003752D
:03004600670A2224
:102D21007F54122EBF7BFF7A117942120CFAD20323
:102D31001216937FF47E011200037F54122EBF7B83
:082D4100FF7A11794C020CFA33
:0B2F1C0075988075A910C298C2992218
:1025A10053D8F8EF540742D8C2DBED24FE60131470
:1025B100601614601914601C2404701C788976401C
:1025C100801678897650801078897660800A7889BB
:1025D1007670800478897680E47888F67889E6F5E3
:1025E100DA20DCFD7888E6248AF8A6D97F037E000C
:1025F100120003788806E6C3940340E07F8A7D03D6
:07260100122ADB788BE6FFD3
:0126080022AF
:102D49008C328D33EF24FE600F1460142402701747
:102D5900121E6EF5C38FC222121E6EF5C58FC422D4
:082D6900121E6EF5C78FC62291
:052F3800D2B4D2B52265
:102E460030020BC2B57FEE7E021200038009C2B4C7
:0C2E56007FEE7E02120003D2B4D2B5223F
:102D98008F328D337F017E00120003D2FEE532258B
:102DA800E054074401788AF608A6337F8A7D021228
:072DB80029D2C2FED2FE2267
:10284900E4FF122EAA7F10122EF47F01122EF47FBC
:1028590012122EF47F04122EF47F08122EF47F1028
:10286900122EF47F15122EF4E4FF122EF47F0812B3
:102879002EAA7F17122EF47F04122EF41228951215
:1028890028957F1D122EF4E4FF022EF47F14122ED8
:06289900F47F04022EF49E
:1017C8007BFF7A117956120CFA7F14122EBF7BFF19
:1017D8007A11796C120CFA753982E4FBFD7FC0121C
:1017E8002198753901753A227B1CE4FD7FC01222CD
:1017F80012753A03753B207B2C7A01E4FD7FC012F9
:101808001D8D7539807B78E4FD7FC012228C30B243
:101818001D121E56121E9FC2021218EC30B22A1256
:1018280018E070021534E535453470F0801B121E3F
:101838005F121E9FD2021218EC20B20D1218E0702F
:10184800021534E535453470F0121E87120003D2B4
:10185800F8E5354534700280FE7F647E001200038F
:101868007E077F447A078A327B448B33E4FD7FC04E
:10187800121E9F753AFD753BD0753C07753D44C2F5
:1018880002AB33AA32E4FD7FC0121A137FE87E034D
:1018980012000374FFF534F53520FF157F0A7E002A
:1018A800120003E535153570021534E535453470F9
:1018B800E8E5354534700280FE121E5F121E9F75E2
:1018C80039FFE4FBFD7FC0122198121E5612230631
:0718D800122E947E007F0038
:1018DF00227F017E00120003E535153522E4FD7FDE
:0B18EF00C01220A274FFF534F5352272
:101AFD007BFF7A117980120CFA7F14122EBF7BFFB7
:101B0D007A11796C120CFA753982E4FBFD7FC012E3
:101B1D002198753901753A227B1CE4FD7FC0122294
:101B2D0012753A03753B207B2C7A01E4FD7FC012C0
:101B3D001D8D7539807B78E4FD7FC012228C30B20B
:101B4D0019C202121BB430B2287F06121BC27002DA
:101B5D001532E533453270EE8017D202121BB420D8
:101B6D00B20F7F02121BC270021532E5334532707F
:101B7D00EE121E87120003D2F8E533453270028053
:101B8D00FE7F647E00120003121E5F121E9F7539C8
:101B9D00FFE4FBFD7FC0122198121E561223061280
:061BAD002E947E007F0073
:101BB30022E4FD7FC01220A274FFF532F533227EAA
:091BC30000120003E53315332282
:10211D0030B217C20212217E30B22412218C70020D
:10212D001532E533453270F08015D20212217E2032
:10213D00B20D12218C70021532E533453270F0125A
:10214D001E87120003D2F8E533453270077F201247
:10215D002A1C80FE7F147E00120003121E5F121EC9
:10216D009F7539FFE4FBFD7FC01221987E007F0033
:10217D0022E4FD7FC01220A274FFF532F533227FD9
:0B218D00027E00120003E53315332230
:030023000224CEE6
:1024CE00C0E0C0D075D008309A41301056300F1889
:1024DE00C20FE5996005756F018048756F02E56E54
:1024EE00156E703F156D803BE56E456D600AE56EAD
:1024FE00156E702F156D802B74712570F8A699E5E9
:10250E007060041570801CC2108018E599700F85DC
:10251E00696D856A6E757006D20FD2108005C21075
:0A252E00756F0AC298D0D0D0E032D9
:03004B00022F3D44
:052F3D00D20EC2B93202
:1023F000C202D203A20292041228F2EF6402604ADF
:10240000BF040E1566C3E56664809480500375664C
:1024100001BF080E0566D3E566648094814003E43D
:10242000F566BF0103122D217F40122EBFAF661249
:102430001E4374222FF974133EFA7BFF120CFAE547
:102440006324FF9202122F0280A8E5667014121E08
:102450008E753707753844E4FD7FC0121FA68E6B5A
:022460008F6C7F
:012462002257
:10237B00C203C2041228F2EF6402605CBF041705AB
:10238B006AE56A70020569D394F9E5699401400620
:10239B00756900756A01BF0813E56A156A70021545
:1023AB0069121E7D5006756901756AF9BF0103122A
:1023BB002D217F40122EBF7BFF7A117995856943C2
:1023CB00856A44856945856A46120CFA7FC87E008A
:1023DB00120003122F028098E56324FF92057F0AF7
:0523EB007E00022B4EF4
:10246300C203C2041228F2EF64026052BF040C05D7
:1024730060E560D394054003756005BF080C1560E3
:10248300E560C394015003756001BF0103122D2160
:102493007F40122EBFE56075F006A42444F974133F
:1024A30035F07543FFF54489457BFF7A1179AA120C
:1024B3000CFA7FC87E00120003122F0280A2E5638C
:0B24C30024FF92057F0A7E00022B4ED2
:1026D300856133C202D203A20292041228F2EF648C
:1026E300026047BF040C0561E561D39402400375A2
:1026F3006101BF080C1561E561C394015003756165
:1027030002BF0103122D217F40122EBFE56175F038
:1027130014A42454F9741335F0FA7BFF120CFAE570
:102723006324FF9202122F0280ABE56165336002DE
:0227330080FE26
:012735002281
:10279800C202D203A20292041228F2EF6402604A33
:1027A800EF64046003BF080CE56570047E018002D5
:1027B8007E008E65BF0103122D217F40122EBFE5DA
:1027C8006575F00DA42490F9741335F07544FFF580
:1027D8004589467BFF7A1179B8856543120CFAE57D
:0A27E8006324FF9202122F0280A862
:0127F20022C4
:102C4B00C202D203A20292041228F28F33EF640263
:102C5B0060197F40122EBF7BFF7A1179C1120CFADB
:0B2C6B00E56324FF9202122F0280D7C5
:012C7600223B
:10266F00C202D203A20292041228F2EF6402605354
:10267F00BF040E1567C3E5676480948150037567C7
:10268F0004BF080E0567D3E5676480948440037523
:10269F006701BF0103122D217F40122EBFAF67EFDD
:1026AF003395E0FE7C007D1212066474982FF97446
:1026BF00133EFA7BFF120CFAE56324FF9202122FEE
:0326CF0002809FE7
:0126D20022E5
:10260900C203C2041228F2EF6402604DBF040E0532
:1026190068D3E5686480948F4003E4F568BF080EC9
:102629001568C3E56864809480500375680FBF011D
:1026390003122D217F40122EBF7BFF7A1179D4120C
:102649001E2DFF3395E0F5438F44120CFA7FC87EA7
:1026590000120003122F0280A7E56324FF92057F71
:062669000A7E00022B4E68
:10289F00C202D203A20292041228F2EF6402604233
:1028AF00EF64046003BF080CE56370047E018002CF
:1028BF007E008E63BF0103122D217F40122EBFE5D4
:1028CF0063600B7BFF7A1179E8120CFA80097BFFAA
:1028DF007A1179F2120CFAE56324FF9202122F0299
:0228EF0080B0B7
:0128F10022C4
:10253800C2027F40122EBF7BFF7A1179FC120CFA7F
:10254800E56324FF9202122F02D203A20292041220
:1025580028F2EF64017041756601F569756A0175C5
:10256800600575610275650175670175640A7563B3
:1025780001756803122E287F54122EBF7BFF7A1232
:102588007910120CFAD2031216937FF47E0112000E
:08259800037D147F04122BBC2B
:0125A0002218
:10293D00C2027D147F04122BBCD203A20292041298
:10294D0028F28F33EF6402602B7F40122EBF7F3051
:10295D00122E077543008F447BFF7A12791C120CDF
:10296D00FA7F14122EBF1227F3E56324FF92021291
:0B297D002F0280C57D147F03022BBCDD
:102CF800122E94E4FF122EBF7BFF7A127928120C51
:102D0800FA7F14122EBF7BFF7A127938120CFA124E
:092D18002D717FF0122A1C80FECF
:1018FA00E4F532122E94E4FF122EBF121E41121A80
:10190A00061219F5122F02D203E56324FF9204127C
:10191A0028F2EF640270030219EEBF040A0532E5E9
:10192A0032B40C03E4F532BF080E1532C3E5326453
:10193A00809480500375320BEF640160030219DD55
:10194A007F54122EBF7BFF7A127956120CFAE532B7
:10195A00B40B00505F901966F828287302198702A1
:10196A00198C02199102199602199B0219A00219DF
:10197A00A50219AA0219AF0219B40219B91223F061
:10198A00804712237B8042122463803D1226D38033
:10199A00381227988033122C4B802E12266F8029FA
:1019AA00122609802412289F801F122538801A12B5
:1019BA00293D80157F40122EBF7BFF7A1279621271
:1019CA000CFA7F207E031200037D147F02122BBCC7
:1019DA001219F5E4FF122EBF121E41121A06122F17
:0B19EA00020219117D147F04022BBCC7
:1019F5007F54122EBF7BFF7A12794A120CFA022D00
:0E1A05007174022FF974143EFA7BFF020CFA82
:102A64007F40122EBF7BFF7A127974120CFA7537ED
:102A740007753844121E56121FA68E6B8F6C7F8A00
:102A84007E02120003753707753844121E5F121F49
:0C2A9400A68E6B8F6C7D147F02022BBCA1
:02152D00A9070C
:10152F00E9FB7A00E56724FE60621470030215E19F
:10153F0024026003021640E9C39429500E7C007DFB
:10154F0007121E4FAA06AB07021680E9C394B350C9
:10155F0011EB25E0FFEA33FEEF24CDFBE43EFA0268
:10156F001680E9C394EB50127C007D0B121E4FEFD7
:10157F002482FBEE34FAFA0216807C007D22121EC2
:10158F004FEF2466FBEE34E5FA021680E9C394CCE4
:10159F005012EBAE027802C333CE33CED8F9FBAA8A
:1015AF0006021680E9C394EA5016EBAE027803C325
:1015BF0033CE33CED8F924D0FBEE34FCFA021680AA
:1015CF007C007D27121E4FEF2472FBEE34E0FA02EF
:1015DF001680E9C39426500E7C007D03121E4FAA7D
:1015EF0006AB07021680E9C394BF501DEB24DAFF48
:1015FF00EA34FFFE7C007D09120664EEC313FEEF92
:10160F00132472FBE43EFA8068E9C394D950117C2D
:10161F00007D09121E4FEF246CFBEE34FCFA805153
:10162F007C007D1D121E4FEF2478FBEE34EBFA8009
:10163F0040EB25E0FDEA33FCEBAE027802C333CE7C
:10164F0033CED8F9FF2DFFEE3CCF2BFDEF3AFCEB5D
:10165F00AE027802CEC313CE13D8F92DFDEC3EFCAB
:10166F00EBAE027803CEC313CE13D8F92DFBEC3EAD
:10167F00FAD3EB9444EA940740057E077F4422AEE9
:03168F0002AF03A4
:011692002235
:10078700E4F5237524FA75251E7526FFF528F52946
:10079700F52AF52BF52DF530F531C200C201F587A5
:1007A700F5D0122F2E122F33122F1CD2BED2971232
:1007B7002F38F56FC2031216937E007F077D007BEB
:1007C700007A00797112075BD29CC298D2ACD2B979
:1007D700C2CDD2AF75C81175C3FF75C20075CBFF07
:1007E70075CA0075CDFF75CC0075C108D2021227F6
:1007F70036122849E4FF122EBF7BFF7A127987123F
:100807000CFA7F47122EBF7BFF7A12799A120CFAE5
:100817007F5A122EBF7BFF7A1279A7120CFAD202E7
:10082700122EE47FC47E09120003122E947E007FED
:10083700067D007B007A00799412075B7E007F0EAD
:100847007D007B007A00797A12075BE4F527E412D2
:100857000C7F40FAE4FD7FC0121F2340097BFF7A1B
:100867001279B6122B15D2057FC87E00122B4EC205
:1008770003C2041228F2EF6403702C7F40122EBFCC
:100887007BFF7A1279C7120CFAE4F527D2057F6449
:100897007E00122B4E7F647E001200030527E5279A
:1008A700C3940A40E7801AE561B401051217C880AE
:1008B70003121AFDE5667009121E8E121E98120C9D
:1008C70065D2AED2BEE5266004152680107526FFD8
:1008D700E4F52DF525C202122736122849E52D60C9
:1008E700030209B4752D08FF122EBFAF66EF3395CB
:1008F700E0FE7C007D0712066474F22FF974143E43
:100907007543FFF5448945AC6BAD6CE41200F37B8E
:10091700CD7ACC799478411200518F498E488D4712
:100927008C46754A00852B4B85654C7BFF7A12797F
:10093700D5120CFAE566640170587F40122EBFAFDE
:10094700777E00121E487D331206CBAA06AB07AF8F
:10095700767E00121E487D331206CB8E478F488A5B
:10096700458B467BFF7A1279E7856943856A44128E
:100977000CFA7F14122EBFAF287E00121E487D335B
:100987001206CB8E438F447BFF7A1279FF120CFA43
:10099700801D7F40122EBF7BFF7A137910121E2D08
:1009A700FF3395E0F5438F44120CFA8002152D2092
:1009B7000E03209427D202122EE47524FAC203C232
:1009C700041228F28F23BF0306120C8D122CF8E5B0
:1009D70023B4010B120C8D1218FA8003E4F523AD32
:1009E70060E4FF1225A18F28E4F527E52775F003BA
:1009F700A42494FFC3740695272471F8E6FB7D03AE
:100A0700122E62E52775F003A42494F9E4FAFB7823
:100A17008A7C00FDFE7F031205E67F8A7D03122A8A
:100A2700DB788BE6FF74782527F8A6070527E527E7
:100A3700C3940240B6E5256004152580287F5A1225
:100A47002EBFE56F75F00FA42400F9741535F07506
:100A570043FFF54489457BFF7A11790E120CFA752D
:100A6700251EE4F56FD2AED2BEE566147003020B05
:100A77000D046003020BA4121E2DFD3395E0FC7ECE
:100A8700017F741206CB8F2CE52324FA604824FEDD
:100A9700602624FE604F24FE60502408704FC3E593
:100AA7006C9444E56B940750447E00E56C252CFB61
:100AB700EE356B120C3E8035AF2C7E00D3E56C9F74
:100AC700E56B9E400CE56C9FFBE56B9E120C3E8030
:100AD7001C120C518017121E98121E56121FA68E3A
:100AE7006B8F6C8008120C518003122A64AE6BAFB7
:100AF7006C7C007D0A1206768F64D2017F647E00CB
:100B0700120003020BA4C3E5289529FFE49400FE15
:100B1700122ED2D3EF9401EE64809480400385288F
:100B270029E565601DE529D39577400BAF29121597
:100B37002D8E2E8F2F802CAF7712152D8E2E8F2F67
:100B47008021E529D37878964007AF29120C718068
:100B5700077878E6FF120C717F7A7D07122CCE8E0C
:100B67002E8F2FE56C652F7004E56B652E600A12DA
:100B77001E98AB2FAA2E120C6520000F7879E6D3AA
:100B870094CC4007D200D202122E4630000F78795B
:100B9700E6C394335007C200C202122E46D2AED229
:100BA700BEE5314530600AE53115317040153080BA
:100BB7003CE561146031147034AE6BAF6CE4FCFD3E
:100BC700FBFAF9F8C312070F702330FF207F14FEDA
:100BD70012000330FF17052B12211D8E6B8F6C75CA
:100BE70030177531708006753017753170E4F52749
:100BF700C3740495272471F8E6120C7F40F2E5715F
:100C0700FD7C007B007AFF7F01122D49E5246004FB
:100C17001524801330010BE5667007D202120026F7
:100C2700C201C202122EE4E52D60077F3A7E001250
:070C37000003C2970208C888
:100C3E00FA753707753844E4FD7FC0121FA68E6B18
:100C4E008F6C22753707753844E4FBFAFD7FC012AE
:100C5E001FA68E6B8F6C22E4FD7FC0121FA68E6BBB
:100C6E008F6C2212152DAA06AB077F7A7D07022CF8
:100C7E0077FDAF27122D980527E527C3940422D2BE
:0A0C8E0097D2057F0A7E00022B4E6C
:10000300E4FDEF4E6018EF1F70011E7C66EC600884
:0E0013001CEDF5F0A4FD80F5D2AED2BE80E467
:0100210022BC
:102CA300AD07AC06ED7803CEC313CE13D8F9FDAC54
:102CB300067802CEC313CE13D8F92DFDEE3CFCEDFE
:0B2CC3004C6007ED1D70F81C80F5222E
:02004900002293
:102B4E008E438F44300530D2ECC2EEE54425E0F5DD
:102B5E0044E54333F543E54445436017E5441544E6
:102B6E00700215437FF47E01122CA3B2EBD2AED2CB
:082B7E00BE80E3C2ECC2EB22B1
:101BCC008E108F118C128D13E5127056E513146064
:101BDC00231460331460382403704775122775136F
:101BEC0010E511AE107802CEC313CE13D8F9F5114F
:101BFC008E108045751213751388E510C313F510FC
:101C0C00E51113F51180327512097513C4802A750C
:101C1C0012037513E8E51125E0F511E51033F51005
:101C2C0080177512017513F4E511AE107802C333E9
:101C3C00CE33CED8F9F5118E10D2ECC2EEE51145AB
:101C4C00106017E511151170021510AF13AE1212BA
:0F1C5C002CA3B2EBD2AED2BE80E3C2ECC2EB221D
:102E6200ED14FEEED39400400EEF2E14F8E6FDEFC3
:0B2E72002EF8A6051E80ECA807A603A2
:012E7D002232
:022DBF00A80763
:102DC100E4F516F517FFEFC39D500EE62517F5172D
:102DD100E43516F5160F0880EDED7C00AE16AF1741
:032DE1001206CB0C
:012DE40022CC
:102ADB00ED14FEC3EE64809480402E7D01D3EE6432
:102AEB0080F8ED648098501EEF2DF8E6FCE814F8A2
:102AFB00E6FBD39C400DA903EF2D14F8A604EF2D94
:092B0B00F8A6010D80D71E80CA56
:012B1400229E
:022C7700A907AB
:102C7900ED14FFEFD394004019EF25E02924FEF865
:102C8900E6FC08E6FDEF25E029F8A60408A6051FDD
:092C990080E1A801A60208A603CF
:012CA200220F
:102CCE00E4F532F533FEEEC39D5014A807E6FA087C
:102CDE00E62533F533EA3532F5320E0F0F80E7ED88
:092CEE007C00AE32AF3312067611
:012CF70022BA
:022E7E00A905A4
:102E8000E4FEEEC399500CA807A60208A6030E0F95
:032E90000F80EFC1
:012E9300221C
:042F420000401454E3
:0D2F0F00D2EDD2EDC2ED7F147E00022CA3A6
:102AA000755EFF85E85F43E80FC2ECC2EFD2EED25D
:102AB000ED7F287E00122CA330EB13E55E600F152E
:102AC0005E7F147E00122CA3D2AED2BE80EAC2ED8D
:0A2AD000855FE8E55E6002D322C3D3
:012ADA0022D9
:102DE5008F5DC2EC122AA053E8F0E55DC4540F5480
:102DF5000F42E8122F0F53E8F0E55D540F42E80249
:022E05002F0F8D
:102EBF008F40C2EC122AA0C2EFC2EEE5404480FF61
:032ECF00022DE5EC
:102EAA008F32C2EC122AA0C2EFC2EEE5324440547D
:052EBA007FFF022DE581
:10273600E4F5E83002087F14FE12000380077F01EB
:102746007E0012000375E803122F0F7F057E00122C
:10275600000312278B12278B75E802122F0F7F01B9
:102766007E001200037F28122DE57F0C122DE57FD7
:1027760006122DE57F01122DE57F02122DE57F025F
:102786007E0002000375E803122F0F7F017E000210
:0227960000033E
:102E94007F01122DE57F027E001200037F02122DB6
:062EA400E5E4FF022EBF71
:0E2EF4008F5CD2EFC2EE122DE5C2EFAF5C2272
:102BBC008F348D35122BD9E535600D15357F2012EC
:102BCC002EF4D2AED2BE80EFAF34022BD9EF3395B8
:102BDC00E0FE74412FF582742F3EF583E493FF02DF
:022BEC002EBFFA
:102EE400300204C2968002D2967F017E0002000363
:10004E0002016BEC5D046005E85904700302016166
:10005E0012012C580460F6EC4860F2EC7004FDFEC0
:10006E00FF22C860DB2481C85009C3986002500685
:10007E000201689850CAF582E9294B4A7005AB8295
:10008E0002015775F0007C1A7880C3EF9BEE9AED53
:10009E0099400DC3EF9BFFEE9AFEED99FDE842F0FD
:1000AE00DC23ACF0D0E0FFD0E0FED0E0FDAB822050
:1000BE00E7101BEB60BAEC2CFCEF33FFEE33FEEDDA
:1000CE0033FD020143E803F830E705C0F075F00098
:1000DE00EF2FFFEE33FEED33FD40B830E7C280AABE
:1000EE0075F020800E75F010800575F0087D007E8D
:1000FE00007F003392D530D503120701EC33401048
:10010E00EF33FFEE33FEED33FDEC33FCD5F0ED2295
:0E011E00E5F0247EA2D513CC92E7CDCEFF22D1
:100C9800E5572443F8E60557227840300C0278439C
:100CA800E475F00112072502060C2005EB7F2ED211
:100CB800058018EF540F2490D43440D4FF30090B2A
:100CC800EF24BFB41A0050032461FFE558600215F1
:100CD80058055BE55B7002055A300C0D7840E475E9
:100CE800F001120725EF020652022EF47403D20C0B
:100CF8008003E4C20CF5578B408A418942E4F558D9
:100D0800F55AF55BE55860077F20120CD380F5751E
:100D180059FFC206C205C207C208C20AC20BC20DE9
:100D2800120CA1FF700D300C057F00120CE4AF5BB4
:100D3800AE5A22B4255FC2D5C209120CA1FF24D035
:100D4800B40A00501A75F00A785830D50508B6FF6D
:100D58000106C6A426F620D5047002D20880D9243C
:100D6800CFB41A00EF5004C2E5D209020FD1D2065F
:100D780080C6D20580C0D20780BCD2D580BAD20A3C
:100D880080B47F20120CD32007077401B5580040A7
:100D9800F1120C98FF120CD3020D0CD20DD20B805D
:100DA80095120C98FB120C98FA120C98F94A4B7091
:100DB8000679C87A107BFF20072EE558602A7E0046
:100DC8008E8275830012062560060EEE655970F056
:100DD800C2D5EBC0E0EAC0E0E9C0E0EE121031D0C5
:100DE800E0F9D0E0FAD0E0FB12060CFF60AAEBC0F5
:100DF800E0EAC0E0E9C0E0120CD3D0E02401F9D069
:100E0800E03400FAD0E0FBE5590460DCD559D9801C
:100E180087D20780A212101460F7E55970010412F6
:100E28000176A959600DE559600914F5591210BBEE
:100E3800EF60F3EA30E702F404C3995077EAF42547
:100E4800590430E701E404F559800D12101460C10B
:100E5800EA05592559120176EA7856F630E701E491
:100E6800255904D55904200A0114121031E4C0E0B0
:100E78001210BB7856E6601320E70714F6120CBB75
:100E8800802204F6D0E014C0E07F00120CBBE559C4
:100E98006007120CB21559800B300A03120CB2D03D
:100EA800E0020D0CD0E00480C512101460A0E559D2
:100EB800041201767856EAF6E559200A0260010420
:100EC800240412103174FF04C0E01210BB120CBBD2
:100ED800E559200A026003120CB2D0E0B559E87F48
:100EE80045120CC57856E67F2B30E7047F2DF404B5
:100EF800C0E0120CD3D0E075F00A84C0F0120CBC2C
:100F0800D0E0120CBC020D0C791080027908C20BDB
:100F1800C20D8008D2D5790A8004790AC2D5E5596C
:050F2800047002F55900
:100F2D00E4FAFDFEFF120C98FC7B08200613120C50
:100F3D0098FD7B1030050A120C98FE120C98FF7B61
:100F4D0020EC3382D592D55013C3E43005069FFFB4
:100F5D00E49EFEE42006039DFDE49CFCE4CBF8C278
:100F6D0006EC700CCFCECDCCE824F8F870F38017DA
:100F7D00C3EF33FFEE33FEED33FDEC33FCEB33FB10
:100F8D00994002FB0FD8E9EB300605F8D0E0C448D4
:100F9D00B206C0E00AEC4D4E4F78207B0070C2EADD
:100FAD00B5590040BCC0E0121033D0F0D0E020069F
:100FBD0004C4C0E0C4B206C0F0120CBCD0F0D5F031
:100FCD00EB020D0C1207350DA9530F10580D7A4C6D
:100FDD000D76420F144F0F1C440F1C490D8F430FFC
:100FED0022550E53460EB1450E1D4710E8500D7E8D
:100FFD002D0D822E0DA52B0D86230DA32010D62A87
:10100D000D3E4800000D9DE559B4FF0375590612BC
:10101D000C98FC120C98FD120C98FE120C98FF788F
:10102D004F0201A5790AA2D5200814300A09B9107A
:10103D00020404B9080104A2D5200B0250010420BA
:10104D0007689207B558005034C0E07F203008196A
:10105D007F30A207720B720A500F12108AC207C29C
:10106D000BC20AC20D7F30800F300A03E9C0E012B7
:10107D000CD3300A03D0E0F9D0E0B558CC300A17C4
:10108D007F30B9100C120CD37F583009077F788050
:10109D0003B90803120CD33007057F2D020CD37F43
:1010AD0020200DF87F2B200BF322920780CF7F009D
:1010BD00B407005005244FF8E6FF22286E756C6CBE
:1010CD0029002D50434958D206120C983006F8C20B
:1010DD0006785830D50108F6020D3E120C982403FF
:1010ED00B405004001E49010CF93120CC4743A1271
:0A10FD000CC4D208755804020F104D
:10012C00E9D2E7C933E833F892D5EDD2E7CD33EC19
:07013C0033FC5002B2D52292
:10014300EC30E7100FBF000C0EBE00080DBD00041D
:100153000BEB6014A2D5EB13FCED92E7FD2274FFC9
:10016300FCFDFEFF22E480F8A2D574FF13FC7D8022
:03017300E480EF36
:10017600F920E72824F950037907E4F42402FB1850
:10018600DBFDE624FB5014E9600DE4F618E604F600
:0F019600B40A08E4F6D9F57401F60A22C2D5229C
:1001A500ED33EC3392D5FA602AB4FF33EDC2E77B29
:1001B500FF60067A0179CAE4227A0179D320D50451
:1001C5007A0179CE224E614E002B494E46002D49CB
:1001D5004E4600E47A08F608DAFC7B00740722E84C
:1001E500C0E0ECC0E0EDC0E0EEC0E0EFC0E0EA75D5
:1001F500F010A4CAABF075F04DA42BFBE435F0FC70
:10020500EA2410FAEB34C5FBEC34D9FCEDC2E7FF68
:1002150075F056A4F42411C5F0F434C58FF0A42A62
:10022500E5F03BE43CF620E7141204D6D0E0FFD01D
:10023500E0FED0E0FDD0E0FC1200518014F4041281
:1002450004D6D0E0FFD0E0FED0E0FDD0E0FC120304
:10025500A0D0E0F8E6FAEDD2E7CD33EC332482FB0B
:10026500E4C3CF33CFCE33CECD33CD33DBF37B07F2
:1002750075F00A846004F6081B0AE5F0F6088FF0AD
:10028500740AA4FFACF08EF0740AA42CFEACF050F6
:10029500010C8DF0740AA42CFDE435F0F608DBDEC4
:0302A500740722B9
:1002A800020161E86480F8E933E83360110460F022
:1002B800ED33EC337009E8FCE9FDEAFEEBFF2204BC
:1002C80060DED3EB9FEA9EE99DE8C2E78CF0C2F7B7
:1002D80095F0400CE8CCF8E9CDF9EACEFAEBCFFB83
:1002E80012012C85D0F05804700320D5B3E80470AF
:1002F800075002B2D502016B92D5EC0460F7E4CC4A
:10030800C0E0C398F8603B94186008400DD0E0FB4B
:10031800020143E4FBFAC9FC8028E830E406E4C99A
:10032800FBE4CAFCE830E305E4C9CACBFCE854079F
:100338006010F8C3E913F9EA13FAEB13FBEC13FCAA
:10034800D8F130F52FC3E49CFCEF9BFFEE9AFEED4D
:1003580099FDD0E0FBEF4E4D4C701222DB030201F9
:1003680068EC2CFCEF33FFEE33FEED33FDED30E7A8
:10037800EB020143EF2BFFEE3AFEED39FDD0E0FB37
:1003880050130BBB000302016BED13FDEE13FEEFE0
:0803980013FFEC13FC0201430A
:1003A000EC4D6011E8497017ED33EC3304600DE457
:1003B000FCFFFEFD22E933E8330470F8020161120C
:1003C000012C58046009E4CC24815006285009020D
:1003D000016B284003020168C0E0EB4A7044B98019
:1003E00006D0E0FB020157EF4E701CBD8008EBFF0A
:1003F000EAFEE9FD80EBE98DF0A4FEE5F002048958
:10040000E9CDF9EAFEEBFFEF89F0A4FCE5F0CE8937
:10041000F0A42EFFE435F0CD89F0A42DFEE435F0F4
:100420008067EF4E7005BD80D780C3EF8BF0A4AC22
:10043000F0EE8BF0A42CFCE435F0F8EF8AF0A42C5D
:10044000E5F038FCE433CB8DF0A42CFCE5F03BF870
:10045000EE8AF0A42CFCE5F038F8E433CF89F0A460
:100460002CFCE5F038CF3400CE89F0A42FFFE5F066
:100470003EFEE433C98DF0A42EFEE5F039CD8AF0BE
:10048000A42FFFE5F03EFEE43DFD33D0E0FB500736
:100490000BBB000F02016BEC2CFCEF33FFEE33FEC5
:0604A000ED33FD020143F3
:1004A6003F8000004120000042C80000447A00005E
:1004B600461C400047C35000497424004B189680E0
:1004C6004CBEBC205A0E1BCA6753C21C749DC5AED7
:1004D600FB60065407601C2323120504EB543860A6
:1004E600091204F01204FF1203A0ECF8EDF9EEFA7B
:1004F600EFCB22EB1204FF80F1543803241C900446
:10050600A6FE93FC0EEE93FD0EEE930ECE93FF2207
:03000000021D01DD
:0C1D0100787FE4F6D8FD758199021D483A
:10051600E709F608DFFA8046E709F208DFFA803EC7
:1005260088828C83E709F0A3DFFA8032E309F608B4
:10053600DFFA8078E309F208DFFA807088828C831C
:10054600E309F0A3DFFA806489828A83E0A3F608D0
:10055600DFFA805889828A83E0A3F208DFFA804CAA
:1005660080D280FA80C680D4806980F28033801081
:1005760080A680EA809A80A880DA80E280CA8033EA
:1005860089828A83ECFAE493A3C8C582C8CCC58362
:10059600CCF0A3C8C582C8CCC583CCDFE9DEE78032
:1005A6000D89828A83E493A3F608DFF9ECFAA9F0B1
:1005B600EDFB2289828A83ECFAE0A3C8C582C8CC07
:1005C600C583CCF0A3C8C582C8CCC583CCDFEADE20
:1005D600E880DB89828A83E493A3F208DFF980CC82
:1005E60088F0EF60010E4E60C388F0ED2402B4047B
:1005F6000050B9F582EB2402B4040050AF23234522
:06060600822390056673DB
:10060C00BB010689828A83E0225002E722BBFE02EC
:09061C00E32289828A83E493221F
:10062500BB010CE58229F582E5833AF583E022508A
:1006350006E92582F8E622BBFE06E92582F8E222D4
:0D064500E58229F582E5833AF583E49322EE
:10065200BB010689828A83F0225002F722BBFE0187
:02066200F32281
:10066400EF8DF0A4A8F0CF8CF0A428CE8DF0A42EAA
:02067400FE2264
:10067600BC000BBE0029EF8DF084FFADF022E4CC68
:10068600F875F008EF2FFFEE33FEEC33FCEE9DEC31
:10069600984005FCEE9DFE0FD5F0E9E4CEFD22ED77
:1006A600F8F5F0EE8420D21CFEADF075F008EF2FC1
:1006B600FFED33FD4007985006D5F0F222C398FDB2
:0506C6000FD5F0EA224F
:1006CB00C2D5EC30E709B2D5E4C39DFDE49CFCEE4A
:1006DB0030E715B2D5E4C39FFFE49EFE120676C346
:1006EB00E49DFDE49CFC800312067630D507C3E441
:0606FB009FFFE49EFE22B9
:0E070100C3E49FFFE49EFEE49DFDE49CFC2209
:10070F00EB9FF5F0EA9E42F0E99D42F0EC6480C861
:06071F0064809845F02201
:10072500FAE6FB0808E6F925F0F618E6CA3AF622D5
:10073500D083D082F8E4937012740193700DA3A353
:1007450093F8740193F5828883E473740293686067
:06075500EFA3A3A380DF67
:102ED200C3EE6480948040028007C3E49FFFE49EB7
:022EE200FE22CE
:10075B00EF4E6012EF60010EEDBB010B89828A83B5
:10076B00F0A3DFFCDEFA2289F05007F709DFFCA9C2
:0C077B00F022BBFEFCF309DFFCA9F02219
:101D0D00020787E493A3F8E493A34003F68001F25E
:101D1D0008DFF48029E493A3F85407240CC8C333D7
:101D2D00C4540F4420C8834004F456800146F6DFA6
:101D3D00E4800B0102040810204080902F27E47EE0
:101D4D00019360BCA3FF543F30E509541FFEE4939B
:101D5D00A360010ECF54C025E060A840B8E493A362
:101D6D00FAE493A3F8E493A3C8C582C8CAC583CA8D
:101D7D00F0A3C8C582C8CAC583CADFE9DEE780BE45
:012F2D0000A3
:00000001FF
